:02000000142BBF
:08000800FF00030E8312031335
:10001000A0000A0EA100040EA2008A110A12172BDA
:10002000B108031D1428080009300000FF3E031D1D
:10003000152800000000B10B14280800AA08031DB1
:1000400022280800F9300000000000000000000035
:1000500000000000000000000000000000000000A0
:10006000000000000000FF3E031D232800000000E8
:100070000000000000000000000000000000000080
:100080000000000000000000000000000000AA0BBB
:1000900022280800B301B401B601B701B501351A31
:1000A00008000310B60DB70DAD0DAE0DB30DB40DB8
:1000B00030083402031D5E282F083302031C672812
:1000C0002F08B3023008031CB403B4023614B50A77
:1000D0004F280808B0003012B0123013B013B0101F
:1000E000B0112D0E0F39B1000F303105AF002F18B0
:1000F0003016AF18B0162F193017AF19B017AE0859
:10010000031DB014300888000A30B1001020881593
:100110000A30B100102088110F302D05AF000A30D1
:10012000B10010200808B0003012B0123013B01324
:10013000B010B0112F183016AF18B0162F19301795
:10014000AF19B017AE08031DB014300888000A308C
:10015000B100102088150A30B100102088110A3033
:10016000B100102008008316031308128812081328
:100170008813881088110C308312AA001E20333097
:10018000AD00AE0169200230AA001E203230AD0061
:10019000AE0169200230AA001E202C30AD00AE0155
:1001A00069200230AA001E200630AD00AE01692091
:1001B0000230AA001E200C30AD00AE0169200230D2
:1001C000AA001E200130AD00AE0169200230AA0055
:1001D0001E200230AD00AE0169200230AA001E20B0
:1001E0000800A91F00292D30AD001030AE00692095
:1001F0002808003CAD00A9090318A90A2D08A80089
:100200002808AA002908AB0027302902031D0A2963
:1002100010302802031C3E29A91B3E29B1012A08DF
:10022000AD002B08AE00AB1F1B29AD09AE09AD0A0E
:100230000319AE0AB10A1030AF002730B0004A20CF
:100240003608AC00311C2629AC09AC0A2C08303E1B
:10025000AD001030AE0069202C08003C03183E2988
:1002600010302A02AD002730031C28302B02AE00CC
:100270002D08AA002E08AB00AC032C29033029025C
:10028000031D4429E8302802031C7929A91B792978
:10029000B2012A08AD002B08AE00AB1F5529AD09ED
:1002A000AE09AD0A0319AE0AB20AE830AF00033056
:1002B000B0004A203608B100321C6029B109B10AE9
:1002C0003108AC00303EAD001030AE0069202C0883
:1002D000003C03187929E8302A02AD000330031CE2
:1002E00004302B02AE002D08AA002E08AB00AC0390
:1002F00067292908803AAD0080302D02031D82292C
:1003000064302802031CAF29B2012A08AD002B0873
:10031000AE00AB1F9129AD09AE09AD0A0319AE0AB3
:10032000B20A6430AF00B0014A203608B100321C76
:100330009B29B109B10A3108AC00303EAD00103044
:10034000AE0069202C08003C0318AF2964302A0253
:10035000AD00031CAB032D08AA00AC03A229290899
:10036000803AAD0080302D02031DB8290A302802E2
:10037000031CE529B2012A08AD002B08AE00AB1F13
:10038000C729AD09AE09AD0A0319AE0AB20A0A308F
:10039000AF00B0014A203608B100321CD129B109A2
:1003A000B10A3108AC00303EAD001030AE0069201B
:1003B0002C08003C0318E5290A302A02AD00031C72
:1003C000AB032D08AA00AC03D8292A08303EAD00A3
:1003D0001030AE00692008002808AD001030AE00D3
:1003E00069200800A908031DF8298030A900FA290E
:1003F000C030A90028082907AD00AE0169200230ED
:10040000AA001E200800AA01B301B4012808B10007
:10041000B201AA190800291C132A3108B3070318CE
:10042000B40A3208B407A90C0310B10DB20DAA0A20
:10043000092AFB308316031308058800FB3083125A
:1004400008058800B3203230AA001E20080083125D
:100450000313A8010130A900F2215430A800EC21B7
:100460004530A800EC214330A800EC214830A8001A
:10047000EC212030A800EC213D30A800EC212030F8
:10048000A800EC21A41F602A6830A800EC216F307E
:10049000A800EC217230A800EC217330A800EC21F8
:1004A0002030A800EC217A30A800EC216F30A800A1
:1004B000EC216E30A800EC216530A800EC21882AE0
:1004C0002308873C24080318031DA41B832A6830D3
:1004D000A800EC216F30A800EC217230A800EC21BC
:1004E0007330A800EC212030A800EC217A30A8005D
:1004F000EC216F30A800EC216E30A800EC216530B3
:10050000A800EC21882A2308A8002408A900F120CB
:100510002030A800EC212030A800EC212030A800D9
:10052000EC212030A800EC212030A800EC21203064
:10053000A800EC212030A800EC210800831203134E
:10054000A801A901F2214E30A800EC212030A8001A
:10055000EC213D30A800EC212030A800EC21260839
:10056000A800A901F1202030A800EC212030A8002B
:10057000EC212030A800EC212030A800EC21203014
:10058000A800EC2108000730831603139F00C03039
:1005900081001922053083169F00813083129F004D
:1005A000A701DC3027020318D72AA70AD12A1F1572
:1005B000A5011F19A50AA801A508031D2814A8084C
:1005C000031DD82A1E08A60060302602A8000E309F
:1005D000A90003223308AD003408AE000A30AF0092
:1005E000B0014A203608A3003708A4002308463C7F
:1005F00024080318031DA41B062BEF3083160505E2
:100600008500EF30831205058500112BEF3083162E
:1006100005058500EF3083120505A8001030280479
:1006200085009E222722CA2A8A110A12C32A83120F
:100630000313220E8400210E8A00200E8300FF0E79
:040640007F0E090020
:02400E003A3541
:00000001FF
